:1000000002178D02001A78680207CD021DEEE4780F
:1000100067F622020022E4F5CF223202002943CF04
:1000200010223202002AD295223232020031C295C9
:0A0030002232320200323232323244
:03003B000200368A
:0300430002003781
:03004B0002003878
:1000530002003902039EE86480F8E933E833601153
:100063000460F0ED33EC337009E8FCE9FDEAFEEBE4
:10007300FF220460DED3EB9FEA9EE99DE8C2E78C92
:10008300F0C2F795F0400CE8CCF8E9CDF9EACEFAE6
:10009300EBCFFB12036985D0F05804700320D5B36E
:1000A300E80470075002B2D50203A892D5EC0460AD
:1000B300F7E4CCC0E0C398F8603B94186008400DA7
:1000C300D0E0FB020380E4FBFAC9FC8028E830E4BB
:1000D30006E4C9FBE4CAFCE830E305E4C9CACBFC87
:1000E300E854076010F8C3E913F9EA13FAEB13FBBA
:1000F300EC13FCD8F130F52FC3E49CFCEF9BFFEE2F
:100103009AFEED99FDD0E0FBEF4E4D4C701222DBD1
:10011300030203A5EC2CFCEF33FFEE33FEED33FDBE
:10012300ED30E7EB020380EF2BFFEE3AFEED39FDF6
:10013300D0E0FB50130BBB00030203A8ED13FDEE4D
:1001430013FEEF13FFEC13FC020380EC4D6011E888
:10015300497017ED33EC3304600DE4FCFFFEFD2220
:10016300E933E8330470F802039E1203695804600C
:1001730009E4CC248150062850090203A82840032F
:100183000203A5C0E0EB4A7044B98006D0E0FB024D
:100193000394EF4E701CBD8008EBFFEAFEE9FD807F
:1001A300EBE98DF0A4FEE5F0020237E9CDF9EAFEB2
:1001B300EBFFEF89F0A4FCE5F0CE89F0A42EFFE479
:1001C30035F0CD89F0A42DFEE435F08067EF4E7055
:1001D30005BD80D780C3EF8BF0A4ACF0EE8BF0A409
:1001E3002CFCE435F0F8EF8AF0A42CE5F038FCE4BD
:1001F30033CB8DF0A42CFCE5F03BF8EE8AF0A42C75
:10020300FCE5F038F8E433CF89F0A42CFCE5F038B2
:10021300CF3400CE89F0A42FFFE5F03EFEE433C9CE
:100223008DF0A42EFEE5F039CD8AF0A42FFFE5F082
:100233003EFEE43DFD33D0E0FB50070BBB000F0255
:1002430003A8EC2CFCEF33FFEE33FEED33FD02038A
:10025300800203A8EC5D046005E8590470030203FF
:100263009E120369580460F6EC4860F2EC7004FDDA
:10027300FEFF22C860DB2481C85009C39860025086
:10028300060203A59850CAF582E9294B4A7005ABCB
:100293008202039475F0007C1A7880C3EF9BEE9A78
:1002A300ED99400DC3EF9BFFEE9AFEED99FDE842F9
:1002B300F0DC23ACF0D0E0FFD0E0FED0E0FDAB8279
:1002C30020E7101BEB60BAEC2CFCEF33FFEE33FEA0
:1002D300ED33FD020380E803F830E705C0F075F065
:1002E30000EF2FFFEE33FEED33FD40B830E7C28061
:1002F300AA75F020800E75F010800575F0087D005A
:100303007E007F003392D530D5031206DAEC3340FA
:1003130010EF33FFEE33FEED33FDEC33FCD5F0EDA0
:1003230022E5F0247EA2D513CC92E7CDCEFF22EDB9
:10033300D2E7CD33EC3392D524814006E4FFFEFDB2
:10034300FC22FCE4CFCECDCC24E0501174FF80ED31
:10035300C3CC13CCCD13CDCE13CECF13CF0470F0BB
:1003630030D5DE0206DAE9D2E7C933E833F892D5AD
:10037300EDD2E7CD33EC33FC5002B2D522EC30E7BB
:10038300100FBF000C0EBE00080DBD00040BEB6088
:1003930014A2D5EB13FCED92E7FD2274FFFCFDFEE6
:1003A300FF22E480F8A2D574FF13FC7D80E480EF84
:1003B300E709F608DFFA8046E709F208DFFA803E2C
:1003C30088828C83E709F0A3DFFA8032E309F60819
:1003D300DFFA8078E309F208DFFA807088828C8381
:1003E300E309F0A3DFFA806489828A83E0A3F60835
:1003F300DFFA805889828A83E0A3F208DFFA804C0F
:1004030080D280FA80C680D4806980F280338010E5
:1004130080A680EA809A80A880DA80E280CA80334E
:1004230089828A83ECFAE493A3C8C582C8CCC583C6
:10043300CCF0A3C8C582C8CCC583CCDFE9DEE78096
:100443000D89828A83E493A3F608DFF9ECFAA9F015
:10045300EDFB2289828A83ECFAE0A3C8C582C8CC6B
:10046300C583CCF0A3C8C582C8CCC583CCDFEADE84
:10047300E880DB89828A83E493A3F208DFF980CCE6
:1004830088F0EF60010E4E60C388F0ED2402B404DF
:100493000050B9F582EB2402B4040050AF23234586
:1004A300822390040373BB010689828A83E022506E
:1004B30002E722BBFE02E32289828A83E49322BB02
:1004C300010CE58229F582E5833AF583E0225006A3
:1004D300E92582F8E622BBFE06E92582F8E222E559
:1004E3008229F582E5833AF583E49322BB010689E9
:1004F300828A83F0225002F722BBFE01F322F8BB6B
:10050300010DE58229F582E5833AF583E8F022506F
:1005130006E92582C8F622BBFE05E92582C8F22238
:10052300EF8DF0A4A8F0CF8CF0A428CE8DF0A42EEC
:10053300FE22BC000BBE0029EF8DF084FFADF0223C
:10054300E4CCF875F008EF2FFFEE33FEEC33FCEE4E
:100553009DEC984005FCEE9DFE0FD5F0E9E4CEFD41
:1005630022EDF8F5F0EE8420D21CFEADF075F00814
:10057300EF2FFFED33FD4007985006D5F0F222C36D
:1005830098FD0FD5F0EA22BB010A89828A83E0F540
:10059300F0A3E022500687F009E71922BBFE07E328
:1005A300F5F009E3192289828A83E493F5F0740153
:1005B3009322BB0110E58229F582E5833AF583E0B6
:1005C300F5F0A3E0225009E92582F886F008E62237
:1005D300BBFE0AE92582F8E2F5F008E222E5832A68
:1005E300F583E993F5F0A3E99322BB010A89828A93
:1005F30083F0E5F0A3F0225006F709A7F01922BB18
:10060300FE06F3E5F009F3192275F008758200EF91
:100613002FFFEE33FECD33CDCC33CCC58233C58231
:100623009BED9AEC99E58298400CF582EE9BFEEDEA
:100633009AFDEC99FC0FD5F0D6E4CEFBE4CDFAE4B9
:10064300CCF9A88222B800C1B90059BA002DEC8BAD
:10065300F084CFCECDFCE5F0CBF97818EF2FFFEE89
:1006630033FEED33FDEC33FCEB33FB10D703994042
:1006730004EB99FB0FD8E5E4F9FA227818EF2FFF82
:10068300EE33FEED33FDEC33FCC933C910D7059BC4
:10069300E99A4007EC9BFCE99AF90FD8E0E4C9FA20
:1006A300E4CCFB2275F010EF2FFFEE33FEED33FDAC
:1006B300CC33CCC833C810D7079BEC9AE899400ACF
:1006C300ED9BFDEC9AFCE899F80FD5F0DAE4CDFB4D
:1006D300E4CCFAE4C8F922C3E49FFFE49EFEE49D60
:1006E300FDE49CFC22EB9FF5F0EA9E42F0E99D427B
:1006F300F0EC6480C864809845F022EB9FF5F0EA43
:100703009E42F0E99D42F0E89C45F022BB01078937
:10071300828A83020AFC5005E9F80207CDBBFE0575
:10072300E9F8020B0889828A83020B14BB010DE5E9
:100733008229F582E5833AF583020AFC5007E9250D
:1007430082F80207CDBBFE07E92582F8020B08E514
:100753008229F582E5833AF583020B14BB010789ED
:10076300828A830208355005E9F8020829BBFE0591
:10077300E9F8020BCF22BB010DE58229F582E5835F
:100783003AF5830208355007E92582F8020829BBA8
:10079300FE07E92582F8020BCF22BB010DE5822972
:1007A300F582E5833AF583020B835007E92582F846
:1007B300020B63BBFE07E92582F8020BB8E5822929
:1007C300F582E5833AF583020B14E6FC08E6FD089F
:1007D300E6FE08E6FF22BB010789828A83020B310A
:1007E3005005E9F8020B24BBFE05E9F8020B3D892D
:1007F300828A83020B4ABB010DE58229F582E583D8
:100803003AF583020B315007E92582F8020B24BB2A
:10081300FE07E92582F8020B3DE58229F582E5838F
:100823003AF583020B4AECF608EDF608EEF608EF0C
:10083300F622ECF0A3EDF0A3EEF0A3EFF022D083C9
:10084300D082E493F608740193F608740293F608D1
:10085300740393F6740473A8828583F0D083D082E3
:10086300120871120871120871120871E473E4938B
:10087300A3C583C5F0C583C8C582C8F0A3C583C516
:10088300F0C583C8C582C822A42582F582E5F03568
:1008930083F58322BB010DE58229F582E5833AF5D1
:1008A30083020BED5007E92582F8020BDBBBFE0741
:1008B300E92582F8020BFFE58229F582E5833AF503
:1008C30083020C11BB0120E58229F582E5833AF509
:1008D30083D0F0D0E0F8D0E0F9D0E0FAD0E0FBE844
:1008E300C0E0C0F0020BF65018E92582F8D083D09F
:1008F30082D0E0F9D0E0FAD0E0FBC082C083020BE3
:10090300E4BBFE18E92582F8D083D082D0E0F9D089
:10091300E0FAD0E0FBC082C083020C08228A8389FC
:1009230082E473E3F5F009E208B5F06BDFF5806765
:10093300E3F5F009E608B5F05EDFF5805A87F009C4
:10094300E608B5F052DFF6804E87F009E208B5F00D
:1009530046DFF6804288828C8387F009E0A3B5F0F6
:1009630036DFF6803288828C8387F009E493A3B55F
:10097300F025DFF5802188828C83E3F5F009E0A37D
:10098300B5F014DFF5801088828C83E3F5F009E479
:1009930093A3B5F002DFF4020A55808780E98090C3
:1009A30080D4803E8015806E807E809D80B7808D50
:1009B30080A380518074803C020A6189828A83EC1F
:1009C300FAE493F5F0A3C8C582C8CCC583CCE493FD
:1009D300A3C8C582C8CCC583CCB5F076DFE3DEE11E
:1009E300807089828A83E493F5F0A3E208B5F0620C
:1009F300DFF4805E89828A83E0F5F0A3E608B5F030
:100A030051DFF5804D89828A83E0F5F0A3E208B5D2
:100A1300F040DFF5803C89828A83E493F5F0A3E616
:100A230008B5F02EDFF4802A8002805789828A83FA
:100A3300ECFAE493F5F0A3C8C582C8CCC583CCE037
:100A4300A3C8C582C8CCC583CCB5F006DFE4DEE21B
:100A530080007FFFB5F0020F2240027F01228982CE
:100A63008A83ECFAE0F5F0A3C8C582C8CCC583CC71
:100A7300E0A3C8C582C8CCC583CCB5F0D5DFE5DE1D
:100A8300E380CF89828A83ECFAE0F5F0A3C8C582BC
:100A9300C8CCC583CCE493A3C8C582C8CCC583CCDA
:100AA300B5F0AFDFE4DEE280A988F0EF60010E4E1F
:100AB30060ABED2402B404005098F582EB2402B439
:100AC3000400508E232345822390099D73EF4E60CB
:100AD30012EF60010EEDBB010B89828A83F0A3DF65
:100AE300FCDEFA2289F05007F709DFFCA9F022BBEC
:100AF300FEFCF309DFFCA9F022E0FCA3E0FDA3E088
:100B0300FEA3E0FF22E2FC08E2FD08E2FE08E2FFAA
:100B130022E493FC740193FD740293FE740393FF28
:100B230022E6FB08E6F908E6FA08E6CBF822E0F845
:100B3300A3E0F9A3E0FAA3E0FB22E2FB08E2F90851
:100B4300E2FA08E2CBF822E493F8740193F9740211
:100B530093FA740393FB227401FF3395E0FEFDFCCB
:100B6300080808E62FFFF618E63EFEF618E63DFDF8
:100B7300F618E63CFCF6227401FF3395E0FEFDFC1B
:100B8300A3A3A3E02FFFF0E582158270021583E093
:100B93003EFEF0E582158270021583E03DFDF0E52F
:100BA30082158270021583E03CFCF0227401FF334E
:100BB30095E0FEFDFC080808E22FFFF218E23EFE76
:100BC300F218E23DFDF218E23CFCF222ECF208EDF1
:100BD300F208EEF208EFF222E6FB08E6FA08E6F97D
:100BE30022EBF608EAF608E9F622E0FBA3E0FAA313
:100BF300E0F922EBF0A3EAF0A3E9F022E2FB08E23A
:100C0300FA08E2F922EBF208EAF208E9F222E493A5
:100C1300FB740193FA740293F9228B218A228923AC
:100C230078287C007D007BFF7A2679767E007F081A
:100C3300120483E4F530F531F530E53025E025E0A5
:100C43002428F8120841DEADBEEF0530E530B402CA
:100C5300E912226200752501752600752700E4F567
:100C630024AB25AA26A92775F014E524A4F58285CB
:100C7300F0831204C27003020E13E52475F014A46A
:100C830029F9EA35F0FA90000A7FFF7EFF7DFF7CA9
:100C9300FF12079DE4FBFAF9F8C31206E8500302BA
:100CA3000E13E52475F014A4FFAEF0AB252527F948
:100CB300E5263EFA9000041204C214605414700333
:100CC300020D5B24026003020DFEAB25AA26A927B1
:100CD30075F014E524A4F58285F083E4120501E997
:100CE3002FF9EA3EFA900001120897E94A4B700384
:100CF300020E13E52475F014A4AB252527F9E52688
:100D030035F0FA90000112089774FF1204EF020EF7
:100D130013AB25AA26A92775F014E524A4F582852B
:100D2300F083E4120501E52475F014A429F9EA35EA
:100D3300F0FA900001120897E94A4B601BE524750D
:100D4300F014A4AB252527F9E52635F0FA90000128
:100D530012089774FF1204EFE52475F014A4AB2571
:100D63002527F9E52635F0FAE9240AF9E43AFAC029
:100D730003C002C00112070FC006C007E52475F0C7
:100D830014A42527F9E52635F0FA9000061207F991
:100D9300D007D006EF2BFFEE3AFEED39FDEC38FC21
:100DA300D001D002D00312075FE52475F014A4FF2D
:100DB300AEF0AB252527F9E5263EFA90000E120882
:100DC30097E94A4B604AAB25E5272FF9E5263EFA1A
:100DD300900011120897C003C002C001AB25E5279C
:100DE3002FF9E5263EFA90000E12089789828A832E
:100DF300D001D002D0031209248015AB25AA26A95D
:100E03002775F014E524A4F58285F083E412050127
:100E13000524E524C394025003020C64E4F530E591
:100E23003025E025E02428F81207CD7BEF7ABE7940
:100E3300AD78DEC31206FE60030080FD0530E530A9
:100E4300B402DC7F0022E4F512F5137514040012DA
:100E53001F20E4F513E513C395144003020FAAE51D
:100E63001375F011A42428F582E43400F583E070AF
:100E730003020FA5E51375F011A4242CF582E434C5
:100E830000F583C083C082E0FCA3E0FDA3E0FEA3E2
:100E9300E0FFC0077867E6FBD007C3EF9BFFEE9444
:100EA30000FEED9400FDEC9400FCD082D083120888
:100EB30035E51375F011A4242CF582E43400F58391
:100EC300E0FCA3E0FDA3E0FEA3E0FFE4FBFAF9F8F6
:100ED300C31206E85003020FA4E51375F011A4240E
:100EE3002CF582E43400F583C083C082E0FCA3E0E8
:100EF300FDA3E0FEA3E0FFE51375F011A42430F594
:100F030082E43400F583E0F8A3E0F9A3E0FAA3E078
:100F1300FBEF2BFFEE3AFEED39FDEC38FCD082D02F
:100F230083120835E51375F011A42429F582E434FE
:100F330000F583E07011E51375F011A42428F58200
:100F4300E43400F583E4F0E51375F011A42434F5DB
:100F530082E43400F583E0FBA3E0FAA3E04A4B60AC
:100F630040E51375F011A42434F582E43400F583CD
:100F7300E0FBA3E0FAA3E08B158A16F517E51375DA
:100F8300F011A42437F9740035F0751801F51989A7
:100F93001A00AB18FA8517828516831209248F125B
:100FA30000000513020E58E47867F6228F169000AE
:100FB300DB7401F0A37400F0A37400F0E4F5219056
:100FC30000DBE0FBA3E0FAA3E0F975F014E521A44C
:100FD300F58285F0831204C260030210E7E516244C
:100FE300FD501F80009000DBE0FBA3E0FAA3E0F9D3
:100FF30075F014E521A4F58285F083E41205017FE1
:10100300FF22AF1AAE19AD18AC17C006C007E52111
:1010130075F014A4FF9000DBE0FBA3E0FAA3E02F3C
:10102300F9EA35F0FA900006D007D006120779AF37
:101033001AAE19AD18AC17C006C007E52175F01438
:10104300A4FF9000DBE0FBA3E0FAA3E02FF9EA356D
:10105300F0FA90000AD007D006120779AB1BAA1C3E
:10106300A91DC003C002C001E52175F014A4FFAEA1
:10107300F09000DBE0FBA3E0FAA3E02FF9EA3EFAED
:1010830090000E1208C79000DBE0FBA3E0FAA3E098
:101093002FF9EA3EFA900004E5161205019000DBF1
:1010A300E0FBA3E0FAA3E0F975F014E521A4F582CF
:1010B30085F0837401120501AB1EAA1FA920C0038A
:1010C300C002C001E52175F014A4FF9000DBE0FB32
:1010D300A3E0FAA3E02FF9EA35F0FA900011120821
:1010E300C7AF21220521E52164026003020FC27FFD
:1010F300FF228D559000041204C2547FF5569000D0
:10110300051204C2F5579000021204C2FE900003B8
:101113001204C2FDEDFF9000071204C2FD9000947B
:10112300E020E113900088EEF0A3EFF0900087ED4C
:10113300F09000867404F0900088E06E7003A3E0E2
:101143006F600302122AE55624FE70030211CF24B6
:10115300FD70030211F414700302121924056003D5
:1011630002121F9000041204C230E7099000AB740E
:1011730003F002121FE557B413099000AB740AF091
:1011830002121FE557B412099000AB740BF0021260
:101193001FE557B414089000AB7402F0807EE55746
:1011A300C39409500B9000987401F09000878069F4
:1011B300E557D3940A4065E5579412505FE49000D5
:1011C30098F0E55724F7900087F08050855758AF83
:1011D300587E00E4F562F56175607F755F437D6855
:1011E3007C01121F657559008F5A90009CEFF080A7
:1011F3002B7B64E4FDAF5712246C8F587E00E4F51B
:1012030062F5617560C8755F427DFFFC121F6590D2
:10121300009AEFF0800690009FE557F0900096E566
:1012230056F0A3E557F0002253DA7FEF24FE603E29
:1012330024FE605824FC607124F870030212CB244E
:10124300F070030212E524E07003021303243F60ED
:101253000302131FED5403FFE5D454FC4FF5D4AE42
:1012630004ED7802CEC313CE13D8F9F5D522ED548D
:101273000325E025E0FFE5D454F34FF5D4AE04EDA8
:101283007802CEC313CE13D8F9F5D622ED5403C496
:1012930054F0FFE5D454CF4FF5D4AE04ED7802CE2D
:1012A300C313CE13D8F9F5D722ED5403C433335403
:1012B300C0FFE5D4543F4FF5D4AE04ED7802CEC35E
:1012C30013CE13D8F9F5DC22ED5403FFE5DB54FC10
:1012D3004FF5DBAE04ED7802CEC313CE13D8F9F588
:1012E300DD22ED540325E025E0FFE5DB54F34FF564
:1012F300DBAE04ED7802CEC313CE13D8F9F5DE22AC
:10130300ED5403C454F0FFE5DB54CF4FF5DBAE04DB
:10131300ED7802CEC313CE13D8F9F5DF22E4F50836
:10132300F509F50A1221501222D675091BE4F50AB4
:10133300E50AC395095039E50A75F003A424BAF503
:1013430082E43425F583E493F50BE50A75F003A4F1
:1013530024BBF582E43425F583E493F50C740193FF
:10136300F50D00FDAC0CAF0B12255E00050A80C025
:101373007F017E007D007C001223DAE4F50AE50A92
:10138300C395095043E50A75F003A424BAF582E432
:101393003425F583E493F50DFF12231C8E0B8F0C7C
:1013A300E50A75F003A424BBF582E43425F58374C0
:1013B3000193650C7004E493650B6007009000E6ED
:1013C300E004F000050A80B67F017E007D007C000A
:1013D3001223DA1222B09000E6EFF0601C7F0312B2
:1013E300231C8E0B8F0C7F0612231C8E0D8F0E7FFA
:1013F3000A12231C8E0F8F100000228B398A3A8920
:101403003B753C0900753D0112058AFFE5F0600359
:101413000214C1EF2403602524FD60030214C1E418
:101423009000AFF0A3F09000AFF0A3F0E4F565F502
:1014330066AB39AA3AA93B75F0FD1205ED9000AFF2
:10144300E0FEA3E0FF7C007D0612052374152FF94F
:1014530074263E7541FFF542894375440175450085
:101463007546B275470075480075493C754A647BFB
:10147300007A00796512158FC3EF6480948250025D
:101483008001C350037F002212257AE53CD39400E8
:10149300400B7B017A0079B2AD3C1216EB00900051
:1014A300B0E004F070069000AFE004F0C39000B029
:1014B300E094069000AFE09400500302142FE4F58B
:1014C3003DAB39AA3AA93BF5F01205ED7F03228B18
:1014D300218A2289230075240112058AFFE5F06021
:1014E3000302157EEF2450603424FA606224B66050
:1014F3000302157EE4F5F01205ED7B017A00796CA9
:101503007F647E007D007C001223C27F0112241CB5
:10151300AB21AA22A923E475F0B01205ED7B017A71
:1015230000796C121D9FEF7002FF22007B017A008D
:10153300796C7F847E037D007C001223C2E4FF125A
:10154300241CAB21AA22A923E475F0B61205ED7B76
:10155300017A00796C121D9FEF7002FF2200900048
:10156300AEE014F0E070937F01121AF3AB21AA22CC
:10157300A923E4F5F01205ED7F0222E4F524AB2163
:10158300AA22A923F5F01205ED7F03228B3E8A3FA1
:10159300894000754B0112058A600302162EE5F09F
:1015A300600302162EE4786CF600AB41AA42A9430D
:1015B300121E89AB47AA48A949E41204EF007FC869
:1015C3007E001220B912259DEF60437552007553BA
:1015D3000075544D7B007A00794C7F30121FDFE594
:1015E3004C20E733AB44AA45A9467F32121E3CABDD
:1015F30047AA48A949EF1204EFAB47AA48A94912E1
:1016030004A9FDAB44AA45A94612220D8009786CB2
:1016130006E6D3954A400FAB3EAA3FA940E4F5F056
:101623001205ED7F022212257A8092E4F54BAB3E40
:10163300AA3FA940F5F01205ED7F03224100C20045
:101643004100C6004A00C70000000000000000007F
:10165300004100C3004100C4004100C5FF4100D167
:10166300004100AE000164FF0163006044002801F3
:101673000100000000006400000001FF0C1D0000D9
:10168300000101000000000C0000000AFF14D2005A
:1016930000010102000000006700000064FF251C38
:1016A3000000010103000000003600000032FF18B3
:1016B3002700000167000468000000004100E5FF07
:1016C3004100E4FF4100E6005000B2EEB981219EE3
:1016D3007C5A600D00000000000000016C00420015
:1016E300AF00004100B1FF008B3E8A3F89408D412E
:1016F300E4F542F543F544F545F546F547FFFEFDB0
:10170300FC1225A590260DE493FE740193FF902609
:101713000BE493FC740193FD1224B71225A5122543
:101723008CE4F542F543E54325E0FFE54233FE74DF
:101733000F2FF58274263EF583E493F546740193E7
:10174300F547AB3EAA3FA94085464CF54DAD411246
:10175300204E00000012259DEF70030080F700006B
:10176300000543E54370020542C39403E542940038
:1017730040B40545E5457002054400C39421E544A2
:101783009400409DE4F544F5452278FFE4F6D8FD46
:101793009000007F007E01E4F0A3DFFCDEFA758198
:1017A3006E0217E2022554E493A3F8E493A34003E3
:1017B300F68001F208DFF48029E493A3F8540724A8
:1017C3000CC8C333C4540F4420C8834004F4568068
:1017D3000146F6DFE4800B010204081020408090EC
:1017E300163FE47E019360BCA3FF543F30E50954E8
:1017F3001FFEE493A360010ECF54C025E060A84010
:10180300B8E493A3FAE493A3F8E493A3C8C582C806
:10181300CAC583CAF0A3C8C582C8CAC583CADFE9DB
:10182300DEE780BE8B218A2289237F021224C9002E
:10183300530702EF604A9000C2E06F600CEFF0E4E0
:101843009000C6F07D64FC806C9000C6E004F0E07C
:10185300D394044065E4F09000C3E0FE24C7F5820E
:10186300E43400F583EFF0EE2401FFE433FE7C0063
:101873007D0A1205359000C3EDF07D327C00803582
:101883009000C6E0D394024031E4F09000C2E0FF40
:10189300A3E0FE24C7F582E43400F583EFF0EE24E1
:1018A30001FFE433FE7C007D0A1205359000C3ED91
:1018B300F07D647C007F011225AD7F00228F5A7971
:1018C300FFE4FBFA90002A75F011EB12088BEA751E
:1018D300F011A42583F583E0655A7068900028759C
:1018E300F011EB12088BEA75F011A42583F583E060
:1018F300704E90002875F011EB12088BEA75F01109
:10190300A42583F5837401F0AF5EAE5DAD5CAC5B83
:1019130090003075F011EB12088BEA75F011A425D5
:1019230083F58312083590002C75F011EB12088BA8
:10193300EA75F011A42583F58312085A000000000C
:10194300E4F9800E0BBB00010AEB64044A60030256
:1019530018C7AF01228B5A8A5B895C1204A9FFC3A3
:10196300648094825003BFFF037FFF22EFFD339512
:10197300E0FC90000075F014ED12088BEC75F01488
:10198300A42583F583E4F090000175F014ED1208AB
:101993008BEC75F014A42583F583E0FBA3E0FAA395
:1019A300E04A4B6039EF75F014A42401F582E43466
:1019B30000F583E0FBA3E0FAA3E0F974FF1204EF60
:1019C300EF3395E0FE90000175F014EF12088BEEF3
:1019D30075F014A42583F583E4F0A3F0A3F0AB5AC8
:1019E300AA5BA95C74FF1204EF7F00228F558D560A
:1019F300E55675F009A42474F9740035F0FA7B01F7
:101A0300C001E55575F009A42474F9740035F0A8F4
:101A130001FC7D01D0017E007F06120AACE55675FC
:101A2300F009A4247BF582E43400F583E0FEE55558
:101A330075F009A4247BF582E43400F583E0B50650
:101A4300047E0180027E00EF701FEE601C90266D05
:101A5300E493FF900095E0C39F5003E004F07B0004
:101A63007A007900121ED58005E4900095F090006D
:101A730095E0FF2275080075090A7DED7C027F2041
:101A830012238F7D017F011225337D017F021225F1
:101A9300337D017F041225337D017F081225337DB9
:101AA300017F10122533E4FD7F0112253EE4FD7F03
:101AB3000212253EE4FD7F0412253EE4FD7F081259
:101AC300253EE4FD7F1012253E7F01122549E4F5F2
:101AD3000AF50BAF0BAD09AC08122568050BE50B36
:101AE3007002050AC39405E50A6480948040E422E9
:101AF3008F2574FFF526F527E4F52BF52AF529F54F
:101B030028E47F04FEFDFCAB2BAA2AA929A828C33D
:101B13001206FE504F90002A75F011E52B12088B28
:101B2300E52A75F011A42583F583E0B5251F852AE1
:101B330026852B2790002875F011E52B12088BE5DD
:101B43002A75F011A42583F583E4F08017E52B248F
:101B530001F52BE4352AF52AE43529F529E435285E
:101B6300F528809DAF27228B508A5189521220ED90
:101B73008F537E01AB50AA51A9521204A9FFC394FB
:101B8300544009EF94D450047F8080027F001204F4
:101B9300A95403FDEE25E025E02435F582E434263F
:101BA300F583E5822DF582E43583F583E4932FF500
:101BB300578E827583001204C2FFAB53E4FD1225D6
:101BC3000FAB50AA51A9528E82758300EF12050103
:101BD3000EBE09A02278087C007D007BFF7A26795F
:101BE3006E7E007F08120483E4F510F511F510E50D
:101BF3001025E025E02408F8120841DEADBEEF050C
:101C030010E510B402E9007867E6700512244480F9
:101C130004120E4900E4F510E510C3940250E8E500
:101C23001025E025E02408F81207CD7BEF7ABE7972
:101C3300AD78DEC31206FE60030080FD051080D878
:101C4300EF701CEB7006EDF4529A529BBB0107ED4B
:101C5300F4529AED429BEB64027043ED429A22EFF9
:101C63006401701CEB7006EDF452915292BB0107B4
:101C7300EDF45291ED4292EB64027022ED42912217
:101C8300EF64027019EB7006EDF452A152A2BB018E
:101C930007EDF452A1ED42A2BB0203ED42A1228B58
:101CA300508A5189528D53E563045401F554E55329
:101CB300F582758300E56375F009A42474F9740053
:101CC30035F0A801FC7D01A9527E00AF8212048386
:101CD300AD54AF63122018EF7019AD54AF631219EE
:101CE300EF0563536301AB50AA51A952AD531210D0
:101CF300F580010000228B088A09890AAF05850F48
:101D03001A850E19850D18850C1785101B85111C56
:101D130085121D85131E85141F851520120FAFEF25
:101D2300FD3395E0FC90000175F014ED12088BEC87
:101D330075F014A42583F583E508F0A3E509F0A362
:101D4300E50AF0AB08AA09F9EF0204EF8F5CE4F5AA
:101D53005DA2AF33F55FC2AFC29412257AE4F55E9C
:101D6300E55CC330E701D39293D29412257AC294EF
:101D7300E55C25E0F55CE55D25E0F55D12257AA2DD
:101D830092E433425D055EE55EC3940840D2C2949B
:101D930012257AE55F24FF92AFAF5D228B258A2659
:101DA30089271200068F2B8E2A8D298C28AB25AA12
:101DB30026A9271207D9C3E52B9BF52FE52A9AF508
:101DC3002EE52999F52DE52898F52CAB25AA26A90A
:101DD3002790000412072FAB2FAA2EA92DA82CC3DE
:101DE3001206FE7F0040027F010022C0E0C0F0C067
:101DF30083C082C0D075D000C000C001C002C00340
:101E0300C004C005C006C007AF8AEF2418FFE4343E
:101E1300FCFEC28DAD07EDF58A8E8C122374D007BC
:101E2300D006D005D004D003D002D001D000D0D04A
:101E3300D082D083D0F0D0E0328F4E8B4F8A50893E
:101E43005112002EE54E4480FF121D4F7FFF121DDD
:101E53004F8F53E553D3943F400375533FE4F552FB
:101E6300E552C3955350197FFF121D4FAB4FAA5034
:101E7300A951855282758300EF120501055280E056
:101E8300120026AF53229000041205B5F54F85F0DA
:101E93004E9000021205B5F55185F05012058AF5F2
:101EA3005385F052749E254FF54F74F6354EF54E1B
:101EB300E4FBFD7F07122239AD53AC52AF51AE5054
:101EC3001224B712258CE54F4480FBE4FD7F070203
:101ED30022398B578A588959C3E5646480948040BA
:101EE3003B900094E0FF30E111A3E09405402DEF17
:101EF30054FD900094F07F0A8012900095E0C39403
:101F0300034019900094E04402F07F03122430E46C
:101F1300900095F0FB7A007964121958221200069A
:101F23008F1E8E1D8D1C8C1BE4FFFEFDFCAB1EAAB9
:101F33001DA91CA81BC31206FE7023FB7A00791F80
:101F4300120C1D7B007A00791F1214D27B007A00D9
:101F5300791F12251C7B007A00791F121827E4FED3
:101F6300FF228E5B8F5CAE04AF05E41202F9AB6215
:101F7300AA61A960A85F120257C004C005C006C0C9
:101F830007AC5BAD5CE41202F9D003D002D001D000
:101F93000012014EE4FBFAF9783F12005D020332AE
:101FA3008F4E8B4F8A50895112002EAF4E121D4F08
:101FB300AF52121D4FE4F553E553C395525017AB7F
:101FC3004FAA50A9518553827583001204C2FF1290
:101FD3001D4F055380E212002602257A8F4E8B4F48
:101FE3008A50895112002EE54E4480FF121D4F7F07
:101FF300FF121D4F8F557FFF121D4FAB4FAA50A9E4
:1020030051E5551204EFAB52AA53A954EF1204EF52
:1020130012002600228F55ED75F009A42474F9747B
:102023000035F0FA7B01C001E55575F009A424746D
:10203300F9740035F0A801FC7D01D0017E007F0911
:10204300120AACEF7F0070027F01228B488A498914
:102053004A8D4B749E254DF54D74F6354CF54CE485
:10206300FBFD7F0712223912258CAB48AA49A94AE6
:10207300854B527F32121FA3AB4D7D017F07022296
:10208300398B258A2689278D28E4F529F529E52921
:10209300C395285020AB25AA26A92775F002E52968
:1020A300A4F58285F0831205B5FDACF0AF291225A6
:1020B30068052980D9227C007D0A120535D3EF9467
:1020C30000EE94004006AC06AD0780047C007D0A58
:1020D300AE04AF05EF1FAC0670011E4C600B12255A
:1020E3007A12257A12257A80EB22E4FE1204A9FFE4
:1020F300EF540FFEC394047D0150027D00EF54F0B2
:10210300C4540F2D2406540724046401540FC454EB
:10211300F0FDEE24046402540F4DFF227B027D2068
:102123007F01121C437B027D107F01121C43E4FBE1
:102133007D047F01121C437B027D087F01121C4337
:1021430000D295C294D293D2920002257AE4F5117B
:102153007B027D087F02121C437D087F021223F15C
:102163007B017D407F01121C437D407F0112247F50
:102173007D407F011224078F1112211F00227B0251
:102183007D017F01121C437B027D807F02121C4371
:102193007B027D407F02121C437B027D207F021263
:1021A3001C437B027D107F02121C43021A77122408
:1021B300587B027D017F01121C437B027D807F02DD
:1021C300121C437B027D407F02121C437B027D2055
:1021D3007F02121C437B027D107F02021C4390008E
:1021E300B1E0B4FF24E4750F01F50EF50DF50C75A0
:1021F30010FF7511247512D8F513F514F5157B012D
:102203007A0079B17D02121CF9228D4EE54E6409E4
:102213007021AF4EFE78DB7C007D011204837B01CD
:102223007A0079DB121B6A7B017A0079DBAD4E12EF
:102233001CA200AF4E228F568D578B5812002E12C0
:10224300257AAF56121D4F8F59AF57121D4F8F5A14
:10225300AF58121D4F8F5B12002612257A002212EF
:1022630000068F358E348D338C32E4FFFEFDFCABDC
:1022730035AA34A933A832C31206FE7006FBFAF955
:102283001224D8E4FEFF227E007F287D007B017AA2
:10229300007900120AD0E4FFEF75F014A42400F5CE
:1022A30082E43400F583E4F00FBF02EC22E4F5117D
:1022B300FF12231C8E128F137F0112231CE513B40C
:1022C300E00EE512B46F09BE5606BF810375110116
:1022D300AF11227D087F021223F17F647E007D000F
:1022E3007C001223DA7D087F0212247F7F647E0044
:1022F3007D007C000223DAE4750F10750E27F50DBF
:10230300F50CF510F511F512F513F514F515FB7A27
:10231300007964FD121CF90022E4FDFCF5527553AB
:1023230000755415FB7A007914121FDFAD14EDFC10
:10233300E515FDAE04AF05221224927D01E4FF12E0
:1023430023587F187EFC122502E4FD7F011224A589
:102353007F01022583EF7005538EFE8006BF0103C4
:10236300438E01BD01045389FB22BD02034389044B
:102373002278681207CDEF2401FFE43EFEE43DFD21
:10238300E43CFC786812082978670622ED5403FEC2
:10239300E5D254CC4F4EF5D2AE04ED7802CEC31342
:1023A300CE13D8F9F5D3221225711221B1122528A3
:1023B3001225B41224F512218112000E0222FA8B87
:1023C300258A268927900004120779120006AB2577
:1023D300AA26A92702075F7B007A0079111223C27C
:1023E3007B007A007911121D9FEF60F40022EF70D9
:1023F30004EDF45280BF0104EDF45290BF0204EDEA
:10240300F452A022EF7005E5805DFF22BF0105E5D0
:10241300905DFF22E5A05DFF22EF7BFF60067A2639
:10242300796380047A2679597D050220849000AE71
:10243300EFF0E4755E0AF55DF55CF55B7F0102186C
:10244300C0438701000000000000000000000000FE
:102453000000000022E4F59AF591F5A1F59BF592B1
:10246300F5A2F5A0F590F58022E4FEEFC39D50029E
:10247300AE05EFD39B4002AE03AF0622EF7003ED30
:102483004280BF0103ED4290BF0203ED42A02253FD
:1024930089F05388CD538EFEE4F58CF58AC2A9C228
:1024A300B922EF7004C2A98002D2A9ED7003C2B9A8
:1024B30022D2B9228E548F557F2412255EAD55AC9E
:1024C300547F2702255EEF7003AF8022BF0103AF65
:1024D3009022AFA0228B368A3789387B007A007925
:1024E3006D0213FE75FEC1EF700453FF7F2243FF9D
:1024F30080221200167F011224E7E4FF0225955380
:1025030089FC438901AD078D8A8E8C22C3EF9557D1
:10251300FFEB6207C3EF9DFF228B218A22892312DF
:10252300001E7F00227B017D027F02121C430022DA
:10253300EFBD010342DA22F452DA22EFBD01034276
:10254300D122F452D122EF600443D2802253D27FAE
:10255300221223AA121BD8E4FEFF22AB05AA04EA27
:10256300FDEB022239EF90267E93FF02122B1222FB
:102573008A12233BD2AF2200000000000000002299
:10258300EF7003C28C22D28C227B807D807F340249
:102593002239E5CF54F84FF5CF22E4FF7D400F02F7
:1025A3002407E4FBFD7F070222398F248C258D2627
:1025B300221213200221E1006FE001568102661707
:1025C300049CC905663707004C086C900948000B4A
:1025D30000080D48BD1600FF1800671A19E01B1309
:1025E30001204800213FC722200023030024723624
:1025F30027180928440229B0002AFDB02C01012D17
:1026030001520000000000007236180909710985A3
:10261300099972361809096A147A258B096B72367F
:1026230018090989147A258B098A7236180909A8A9
:10263300147A258B09A9451F145C2BC9E3116D5F1F
:102643008A2BAF031DF31AE2F0D104D87142AF0411
:10265300DD07611338640000000000000000000083
:1026630000FF00FF00FF00FF00FF07000000000065
:102673000000000000000000000000010204081038
:012683002036
:00000001FF
